:1000000020C03CC03BC03AC039C038C037C036C041
:1000100035C034C033C032C031C030C02FC003142B
:100020006EE6FFFFFFFF000000000007385A89FF5F
:1000300001020305060809000204070900F3F4EEB3
:10004000090011241FBECFEDCDBF20E0A0E6B0E037
:1000500001C01D92A537B207E1F7E6E7F0E0128292
:1000600081E08683808788E58187E0E6F0E08DEF98
:1000700087838EEF8583712C9DD06EC1C1CF20ED1B
:1000800037E0019720F0F9013197F1F7FACF0895A1
:1000900088EE93E0F4CF369A3699FECF85B1089575
:1000A000CF93C72D81E0870D8F73782E662D90E05A
:1000B00045D16FEF8C2F90E0CF9140C1FF920F930D
:1000C0001F93CF93DF93F82E07E710E0CEE7D0E041
:1000D000F11005C0CE012AD1F801808304C0F801D7
:1000E0006081CE012BD121970F5F1F4FC537D105FE
:1000F00079F7DF91CF911F910F91FF900895D0DF95
:1001000081E0DCCFCF92DF92EF92FF920F931F93AB
:10011000CF93C82F8B018FE1E82E80E0F82E98E274
:10012000C92E90E0D92ECC2381F0F701849189BDAE
:10013000F601849188BDC801A2DF19BC18BCC801B2
:100140009EDFC8019CDFC150EECFCF911F910F9170
:10015000FF90EF90DF90CF900895CF93DF93D82F4B
:1001600064E170E08AE0CEDF84EF91E088DF8D2FDC
:1001700064E6D0D0CAE06C2FCDD0892F68EC70E057
:10018000C1DF86DF8D2F6C2FC5D0D92FC3D0892F2B
:1001900068EC70E0B7DF7CDF68EC70E08D2FB2DFD9
:1001A00077DF64E170E08AE0ADDF84EF91E0DF911A
:1001B000CF9165CF1092750083EA87B986EC86B936
:1001C0003699FECF369A86B1C82FC07486FDFBCF14
:1001D00085B18095582E712C872D90E0A7D0682E80
:1001E0008F3F31F08FEF68120AC0612C88DF09C0A1
:1001F000872D91E0970D792E803470F3F3CF80E056
:100200005DDF20917E002F5F40E350E0222391F0DC
:10021000CA010196FC013197E491AC2FB0E0A859D6
:10022000BF4FEC93EE2319F0C82FC41BF2CF21501F
:10023000AC01ECCFC093800084E08C0F982F9150DC
:10024000E92FEC1BF0E0E35CFF4FE491A92FB0E055
:10025000A859BF4FEC939C13F2CFE82FF0E0E95977
:10026000FF4F91E0309168002081321390E0891BAC
:1002700080938100962D953FD0F5252D2134B0F443
:10028000809182008F3F29F48091750080938200D5
:1002900006C081E0860D682E8C1708F0612C8091D5
:1002A00082008F5F8F718093820021C090917500D2
:1002B000909382002F3AB8F490917C00992369F0D2
:1002C000962D6C1202C0612C12C0662019F091505C
:1002D000692E0DC08150682E0AC081E0860D682EFF
:1002E0008C1788F704C080917800882361F38FE32E
:1002F00084BB8BE087BB88EF88BB81E083BF81EA4A
:100300008ABD87B986EC86B98CE291E0B8DEC3DE9F
:1003100024DFFACF991B79E004C0991F961708F0E3
:10032000961B881F7A95C9F780950895E199FECFAD
:100330001FBA8EBBE09A99278DB30895262FE199B5
:10034000FECF1CBA1FBA8EBB2DBB0FB6F894E29A33
:0C035000E19A0FBE01960895F894FFCFCB
